:10000000F89411240FEF0DBF00E10EBFA0E0B1E0A6
:10001000C2E1D1E0CA1BDB0B2196E2E0F1E02197BF
:1000200019F005900D92FBCFA2E1B1E0C2E1D1E061
:10003000CA1BDB0B2196219711F01D92FCCF02D039
:100040000C9402F0EF92FF920F931F93CF93DF93E4
:100050000F2EF8E3EF2EFF24F02D02E310E00E94B4
:10006000510080E091E00E9472008FEF87BB83E037
:1000700081BBC0E0D0E0F701C0838D2F992787FDB9
:100080009A958370F801808380E090E00196F5E70F
:1000900080339F07DCF380E191E00E94720021969B
:1000A000EACF109290008FE089B982E08BB988E1A5
:1000B0008AB986E0809395008F9A97988E98969A41
:1000C00008955F9904C097985F9BFECF979A8CB173
:1000D000992787FD909508958699FECF5D9BFCCF6B
:1000E0008CB90895CF93DF93EC018881882331F098
:1000F00089910E946C0088818823D1F7DF91CF918C
:02010000089560
:1001020031302D62697420636F756E7465720A00F6
:020112002E00BD
:00000001FF
